:100000000C9459020C9476020C9476020C947602AD
:100010000C9476020C9476020C9476020C94760280
:100020000C9476020C9476020C9469110C94AB102B
:100030000C9412190C9476020C9476020C947602AD
:100040000C9476020C9476020C9476020C94760250
:100050000C9476020C94C5180C9476020C947602DB
:100060000C9476020C9476020C9476020C94760230
:100070000C9476020C9476020C9476020C94760220
:100080000C9476020C9476020C9476020C94760210
:100090000C9476020C9476020C9476020C94760200
:1000A0000C9476020C9476020C947602A6041A053F
:1000B000AE0478047C04B2047F04B504C0048A044E
:1000C00010058E04C4049204C804F2049604CC04FF
:1000D000FC049C04D204DC048304B9048604BC043C
:1000E000A104D704E80408050A057404AA0423053A
:1000F00049054F053D05430555055B0561055A0654
:100100005A068C068C060B072707280828082C0798
:10011000A007B107B107A90BAC0BDF0BF80BFF0B66
:100120000A0C0D0C0D0C0D0CDA0CDA0C420C440C04
:10013000490C6F0C910C940C970CBA0CBB0EE20E90
:100140009310E20E93102E0F510F9310471057107B
:10015000000000000000000000000000000000009F
:10016000000000000000000000000000000000008F
:10017000000000007E0F00D4FFFFFFC700000078E2
:1001800000000000000000002A2B280000000000F2
:100190000000000000000000000000290000000036
:1001A0002C1E3420212224342627252E362D3738A4
:1001B000271E1F202122232425263333362E3738AD
:1001C0001F0405060708090A0B0C0D0E0F1011126B
:1001D000131415161718191A1B1C1D2F3130232D37
:1001E000350405060708090A0B0C0D0E0F10111235
:1001F000131415161718191A1B1C1D2F3130354CE6
:1002000005010902A10185020901A10005091901E1
:10021000290815002501950875018102050109309D
:1002200009311581257F95027508810609381581E8
:10023000257F950175088106050C0A380215812570
:100240007F950175088106C0C005010980A101855F
:100250000319012AB700150126B700950175108111
:1002600000C0050C0901A101850419012AA002158D
:100270000126A002950175108100C005010906A1A3
:10028000018506050719E029E71500250195087580
:100290000181020507190029EF1500250195F07568
:1002A000018102050819012905950575019102953D
:1002B0000175039101C00660FF0961A10109621582
:1002C0000026FF009520750881020963150026FFAE
:1002D00000952075089102C005010906A1010507D6
:1002E00019E029E71500250195087501810295019E
:1002F000750881010507190029FF150026FF0095E3
:1003000006750881000508190129051500250195C4
:100310000575019102950175039101C009025B0009
:10032000030100A0FA0904000001030101000921F2
:10033000110100012244000705810308000109049E
:100340000100020300000009211101000122220026
:1003500007058203200001070503032000010904AB
:100360000200010300000009211101000122B60072
:100370000705840320000112010002000000082587
:100380004060600100010200011003470068006541
:100390000072006B0069006E000000200334003022
:1003A000002000500065007200630065006E00745C
:1003B00000200043006C0075006200000004030987
:1003C0000414001A000800150017001C0018000C87
:1003D000001200130004001600070009000A000BB9
:1003E000000D000E000F0029001D001B0006001963
:1003F000002A002C00050011001000280001000157
:1004000000010001000100010001000100010001E4
:1004100000010001000100010001000100010001D4
:10042000000100010001000100010001004C000179
:1004300000010001000100010001000100010001B4
:1004400000010001000100010001000100010001A4
:100450000001000100010001000100010001000194
:100460000001000100010001000100010001000184
:100470000001000100010001000100010001000174
:100480000001000100010001000100010001000164
:100490000001000100010001000100010001000154
:1004A0000001000100010001000100010001000144
:1004B000000011241FBECFEFDAE0DEBFCDBF11E098
:1004C000A0E0B1E0EAE0F4E402C005900D92A236AB
:1004D000B107D9F722E0A2E6B1E001C01D92A23532
:1004E000B207E1F70E946F080C9403220C940000FD
:1004F000A8E0B0E0EEE7F2E00C94BF21FC018481BB
:10050000882309F4E8C57F0121E04081518162819F
:10051000738195810E94E21F8C01F70185818823F8
:1005200009F4BAC1980137572038310508F032C1B3
:10053000003108F0E2C28FEF93E00E94EC208111BD
:10054000DCC238E1A32EBB24B394002379F0A114BC
:10055000F4E0BF0609F4D1C2C5010E94EC2081116C
:1005600001C001502FEFA21AB20AEFCFCE010196BF
:100570002C0188E0F20111928A95E9F72AE0322EE7
:1005800085010F5F1F4FC5010E94EC2089831A82ED
:10059000882309F4B2C2813009F041C06501F2E05C
:1005A000CF0ED11CC8010E94EC208A83882309F455
:1005B000A4C29FEF980F933060F423E0A20EB11C09
:1005C000C6010E94EC208B83882309F496C21C820A
:1005D00029C0843031F54E0133E0830E911C02E0D6
:1005E00010E056018FEFA81AB80AC6010E94EC204D
:1005F000F40181934F01882309F47FC28C3741F4C1
:10060000E2E0F0E0EC0FFD1FE00FF11F10820AC0E6
:100610000F5F1F4F65010730110519F76EC25801B2
:1006200001C056018201F8012081222309F4A8CFDC
:10063000213009F053C08181813081F46801F2E0FA
:10064000CF0ED11CF8018281893319F460E570E086
:1006500002C060E070E00E94BD1F15C0823049F406
:100660006801F2E0CF0ED11CF80182810E94061FC2
:100670000AC0833051F46801F2E0CF0ED11CF801BA
:1006800082810E94AC1E860182C0843019F00F5F07
:100690001F4F7DC0F80122810E5F1F4F80E090E068
:1006A00030E0205331092A30310568F4389EA0012A
:1006B000399E500D1124C901840F951F0F5F1F4FE4
:1006C000F8012081EDCF009709F461C0EFE9FFE068
:1006D0003197F1F700C000000197F5CFE22FF0E06D
:1006E000E058FE4F2490822F86958695869590E05F
:1006F000FC01E059FE4F64902770712C022E02C05D
:10070000759467940A94E2F7F1E06F227724FC0174
:10071000E05AFE4F8490912C022E02C0959487944B
:100720000A94E2F731E083229924FC01E05BFE4F5A
:10073000C490D12C02C0D594C7942A95E2F781E0E9
:10074000C822DD246114710419F081EE0E94061F95
:100750008114910419F086EE0E94061F60E070E09B
:10076000822D0E94BD1F8114910419F086EE0E9413
:10077000AC1E6114710419F081EE0E94AC1EC1140C
:10078000D10429F060E070E08CE20E94BD1F0F5F91
:100790001F4F49CF023098E7190709F470C058F489
:1007A0000115F8E71F0791F0013028E7120709F05B
:1007B00073C080E00CC0043038E7130709F446C06A
:1007C00068F00530E8E71E07C9F066C083E00E94C4
:1007D000841C809128020E947E1C8FC18091280277
:1007E000982F96959695969549F1915E990F990F48
:1007F000990F8770892B8093280214C0909128024A
:10080000892F8695869586958F5F8F719770843036
:1008100008F03FC0880F880F880F892B809328022B
:1008200080912802887F91E009F490E0809128026D
:1008300090FB80F9809328020E947E1C8091280200
:100840008695869586950E94DC1B57C120912802CB
:10085000822F869586958695482F50E04330510526
:1008600054F48F5F982F990F990F990F822F8770EB
:10087000892B80932802809128028160DBCF8091B0
:10088000280280FF03C00E949E1C37C10E94AD2039
:1008900034C190932802C4CFF801E851FC47E730F7
:1008A000F10508F4E6C0882309F43BC11092380230
:1008B000980130572332310508F00CC184E090E0F4
:1008C0000E94F4209093400280933F02F801E1508F
:1008D000F047E232F10520F4EA5AFF4F0C949821D8
:1008E00080913F028160ACC0809140028860B4C0BA
:1008F00080913F028260A4C080913F0220C080911D
:100900003F0288609DC0809140021EC080914002DD
:100910008260A2C080913F02806192C080913F02BC
:1009200080628EC080913F0280648AC00E94921DC6
:1009300080913F02806884C080913F02886084601B
:100940007FC0809140028260816086C080913F02BA
:100950008E7F76C080914002877F7EC080913F026B
:100960008D7F6EC080913F0220C080913F02877FC3
:1009700067C0809140021EC0809140028D7F6CC094
:1009800080913F028F7E5CC080913F028F7D58C076
:1009900080913F028F7B54C00E94921D80913F0244
:1009A0008F774EC080913F02877F8B7F49C08091B7
:1009B00040028D7F8E7F50C080913F0282FB2227B4
:1009C00020F991E0922790FB82F990FB83F938C0DF
:1009D00080914002982F909591708E7F892B90FB8B
:1009E00081F93AC080913F0286FB222720F991E0ED
:1009F000922790FB86F924C00E94921D80913F02AD
:100A000087FB222720F991E0922790FB87F918C0F5
:100A100061E001C060E08EE090E00E940A211EC00B
:100A200080913F0284FB222720F991E0922790FBDE
:100A300084F906C080913F02982F909590FB80F931
:100A400080933F020BC08091400283FB222720F954
:100A500091E0922790FB83F98093400260913F02DE
:100A60007091400284E090E00E9428210E94921D33
:100A700044C0E858FF4F0C94982106E221EE41EE65
:100A80006AE17CE723C007E225EE45EE6BE17CE7F7
:100A90001DC006E221EE40EE68E17CE717C007E2E8
:100AA00025EE44EE69E17CE711C006E221EE42EE5C
:100AB0006CE17CE70BC007E225EE46EE6DE17CE7DA
:100AC00005C008E221E045EE6EE17CE7C7010E9427
:100AD000341A13C00631FCE71F0791F58091FA0123
:100AE0008A7A91E009F490E090936401811117C033
:100AF00089E20E9469190E94CC158091CF0187700C
:100B000009F4E9C2F7018581882309F4E4C28091E0
:100B1000400282FFE0C282E00E941E16DCC285E332
:100B2000E8CF06312CE7120709F0BCC280916401BE
:100B3000811104C089E20E943B19DDCF85E3FBCF20
:100B400007373CE7130711F481E0BAC208379CE786
:100B5000190709F4B4C29801205E324520323105EC
:100B6000A8F4811115C00F7181E090E09C0102C0D2
:100B7000220F331F0A95E2F78901622F83E090E08C
:100B80000E940A21802F0E946C1DB7CF8823E9F1B3
:100B900003303CE7130729F148F401159CE71907D6
:100BA00091F00130ECE71E0711F12FC00B35FCE787
:100BB0001F0741F10C352CE71207E1F00A351C47FD
:100BC00021F581E020C00E94921D8FEF94E3ECE0BC
:100BD00081509040E040E1F700C000000E94B4184E
:100BE0008CCF6FEF7FEF80E090E00E9428210E9481
:100BF000972083CF8091400282FB882780F991E083
:100C0000892701C080E00E943516F70185810081A7
:100C10001181882349F0C8010E94AB1CD82E682F8F
:100C2000C8010E941B1D04C0C8010E94E71CD82EE9
:100C3000B8018D2D0E9476140E9484148C01A82E78
:100C4000F701B580968092949FE099228091CF0120
:100C5000877001F1BB20F1F0812F807F803469F033
:100C600080E2800F8830B0F0812F807E803229F4BE
:100C7000F1E0F01778F4992069F08091400282FF4A
:100C800009C082E00E941E168091CF018770DD248A
:100C9000D3948111D12CC12EC2948FE0C8228C2D07
:100CA00090E08C30910508F0D3C1FC01E158FF4F72
:100CB0000C949821812F807F1F70882311F012954A
:100CC000107FBB20B9F0112309F4B0C180E2800F7E
:100CD000883010F0A11006C09091FA01192B1093E2
:100CE000FA0105C09091D101192B1093D1010E94F6
:100CF000CC159CC1802F0E94AC1E112309F4A8C101
:100D0000005E083080F1AA2071F110959091D10118
:100D100019231093D1012AC0812F807F1F70803248
:100D200011F01295107FAA2029F021E0A21609F4F3
:100D30004DC058C08091400282FD1BC0BB2069F0AD
:100D4000112339F03091FA01312B3093FA010E94CE
:100D5000CC1580E00E94061F7BC180E00E94AC1E83
:100D6000112309F475C1812F0E94C5150E94CC156D
:100D70006FC1BB2081F09920C9F131E0931268C1A5
:100D80003091D001812F8323181709F461C1312BD1
:100D90003093D0015DC191105BC1812F0E94C31DB2
:100DA0003091D001812F832329F0812F8095382322
:100DB0003093D00120916501812F822309F448C12D
:100DC000312F309523232093650142C1BB2029F0A8
:100DD00085E0891508F43CC109C094E0991508F430
:100DE00037C115C0BB2031F0911020C1812F0E9466
:100DF000CA1D2EC1992059F0093309F026C1EFEF21
:100E0000F7EE23E0E150F0402040E1F71CC1812FD4
:100E10000E94C31D1DC1812F86958695837019F090
:100E2000813059F015C1BB2019F0C801937002C080
:100E300080E090E00E94C51913C1BB2019F0C801E1
:100E4000937002C080E090E00E94A01909C16B2D50
:100E5000802F0E94D41D04C1812F8370A9F5B11089
:100E6000FBC0402F429546954770440F440F802F9A
:100E70008F7090E09C01042E01C0220F0A94EAF7C3
:100E800004FF08C08FE090E001C0880F4A95EAF7A0
:100E9000809501C080E0169516951370123069F0A8
:100EA00088F490916B01113019F0822B892302C0D4
:100EB000922B892B0E946C1DCFC0822B90916B01CD
:100EC0008927F8CF822BF6CFBB2019F0812F8170B4
:100ED00001C08695882309F4BFC0402F42954695EE
:100EE0004770440F440F802F8F7090E09C01042EB8
:100EF00001C0220F0A94EAF704FF08C08FE090E0D7
:100F000001C0880F4A95EAF7809501C080E01695E8
:100F100016951370123059F078F490916C011130DD
:100F200019F0822B892309C0922B892B06C0822BB2
:100F300090916C01892701C0822B0E94501D8CC0AA
:100F40001F70BB2039F0812F0E94601D802F0E94EE
:100F5000CA1D82C0802F0E94C31D812F0E94531D75
:100F60007BC0802F32EFA31681F13A1538F090EF55
:100F7000A91659F0E1EFAE1619F154C0F3EFAF1610
:100F800059F124EFA216C1F04DC0BB2081F034E02E
:100F9000391508F45DC01F7181E090E0012E01C099
:100FA000880F0A94EAF790916C01892720C085E0A8
:100FB000891508F44DC0EFCF8091400282FD1AC020
:100FC000BB2029F0812F8F7120C0BB20D9F3812F46
:100FD0008F710E94531D3CC0BB2041F01F7181E006
:100FE000012E01C0880F0A94EAF701C080E00E9438
:100FF000501D2EC0BB2061F0812F8F7198E0899F1A
:101000009001112423602093CF010E94601D20C015
:1010100081E00E941E16E1E0E915D0F482E00E9412
:101020001E1616C0BB2021F0992061F2802F92CEAF
:10103000992069F2893349F4FFEF27EE33E0F1504C
:1010400020403040E1F700C00000802F0E94AC1E1D
:1010500088EF8C0D843020F40E94EA190E94D51F7D
:10106000DD20A9F08091CF0180FD11C0F70115822C
:101070008695869586950E94601DC7010E9478021C
:101080008091CF018695869586950E94531D20E01C
:10109000F7014081518162817381848195810E9431
:1010A000E21F19C00737ECE71E0711F481E00BC0FF
:1010B0000837FCE71F0709F04ECD82E004C082E04C
:1010C0000E94601D02C00E94531D43E062E081E067
:1010D0000E94361812CD2896E2E10C94DB21A6E29C
:1010E000B0E0E5E7F8E00C94BF2185B7806885BFE4
:1010F00085B7806885BF84B7877F84BF0FB6F894B3
:10110000A8958091600088618093600010926000D3
:101110000FBE90E080E80FB6F89480936100909342
:1011200061000FBE81E080930D0182E892E190930F
:101130006301809362010E94EF100E940E11809162
:10114000E20084608093E200789480918401882397
:10115000A1F01091E9001F709091EC00892F81702F
:1011600090FD80E8182B1092E9008091E80083FD43
:101170000E94D30D1F701093E90082E084BD93E0BC
:1011800095BD9AEF97BD80936E000E941B1A811146
:1011900002C00E949E1B0EE011E063E1E62E61E0BA
:1011A000F62ED8018D918D018F3F11F00E94B5135D
:1011B000E016F106B1F703E111E059E1E52E51E047
:1011C000F52EF80181918F018F3F11F00E94B51328
:1011D000E016F106B1F785E0E4E7F1E0DF01282F42
:1011E0001D922A95E9F7E6E6F1E0DF011D928A9566
:1011F000E9F780E090E00E94F420853E9E4F21F4C4
:101200000E941B1A811163C065EE7EEF80E090E0C2
:101210000E94282160E082E090E00E940A2181E0A3
:1012200080936B0161E083E090E00E940A2160E01E
:1012300074E184E090E00E94282160E086E090E084
:101240000E940A2160E087E090E00E940A2140E0CD
:1012500050E0BA0188E090E00E941C2160E083E247
:1012600090E00E940A2160E08CE090E00E940A2158
:1012700060E08DE090E00E940A2119821A821B82B0
:101280001C821D821E821F82188648E050E067E1A2
:1012900070E0CE0101960E94FA2040E050E0BA01D1
:1012A0008FE190E00E941C2180E00E94FC190E94C6
:1012B0009E1B40E050E0BA018FE090E00E941C21AC
:1012C00040E050E0BA0183E190E00E941C2182E0FE
:1012D00090E00E94EC2080936D0184E090E00E94F9
:1012E000F4209093400280933F020E94CC13EFEFD2
:1012F000F6E721E0E150F0402040E1F700C00000B7
:101300000E94CC138091740180FF08C06FEF7FEFC3
:1013100080E090E00E9428210E94B41883E090E0D1
:101320000E94EC200E946C1D559A5D9A209A289A82
:10133000259A2D9882E88093800089E1809381002E
:101340008FEF9FEF90938700809386000E94C520C7
:101350000E94C52080E091E090933C0280933B0284
:1013600038E1C32ED12C40E1542EBB24B394AA24DF
:10137000A3948E010F5F1F4F80918401853009F087
:1013800045C080918401853009F038C08091840186
:10139000843041F180E00E94841C80E00E94D51FCF
:1013A0001092410280E40FB6F894A895C0926000B4
:1013B0000FBE8093600083B7817F846083BF83B753
:1013C000816083BF7894889583B78E7F83BF0FB683
:1013D000F894A895809160008861809360001092D5
:1013E00060000FBE0E94CC13E4E7F1E0819181110F
:1013F000EAC291E0E937F907C9F7C3CF0E94921D0D
:101400000E94C5200E94EA190E94D51F0E94CC1399
:101410009EE6E92E91E0F92E24E7822E21E0922E1D
:10142000D401F70191918D91892721E0E337F207EB
:1014300019F08823B9F305C0811103C00E94A115DA
:1014400032C0712CD4012D904D01F701308032242F
:1014500009F1612C44244394832D8421A1F069A2D5
:101460007AA20E9406199CA38BA3ADA291E0822DC3
:10147000842109F490E09EA349A15AA16BA17CA10B
:101480008DA10E9407206394440CF6E06F12E4CF14
:10149000D7012C927394BFEFEB1AFB0AE5E07E12A2
:1014A000D1CF0E94FA1886E0E0E3F2E0D801019083
:1014B0000D928A95E1F77090310290903202F0908F
:1014C0003302E09034028090350210923202109282
:1014D00033021092340210923502911003C0FF20A3
:1014E00009F44BC080912E0290912F020E94EB18BC
:1014F0009C0190912902992309F48BC22531310571
:10150000E0F19F3F19F09F5F90932902992061F0CD
:101510000E94041B191414F491E001C09FEF899FED
:10152000802D112480933202FF2061F00E94041B61
:101530001F1414F09FEF01C091E0899F802D1124AA
:1015400080933302809132028823B9F06090330295
:10155000662099F00E94241B882319F080933202A0
:1015600002C0B0923202862D0E94241B882319F0FB
:101570008093330202C0B0923302E11003C088208E
:1015800009F44BC080912C0290912D020E94EB181F
:101590009C0190912A02992309F440C2213531051A
:1015A000E0F19F3F19F09F5F90932A02EE2061F0D7
:1015B0000E94E21A1E1414F491E001C09FEF899F6B
:1015C000802D112480933402882061F00E94E21A59
:1015D000181414F09FEF01C091E0899F802D112411
:1015E00080933502809134028823B9F060903502EF
:1015F000662099F00E94241B882319F080933402FE
:1016000002C0B0923402862D0E94241B882319F058
:101610008093350202C0B092350280913102871169
:101620001AC080913202882311F0891114C0809170
:101630003302882311F0F8120EC0809135028823FE
:1016400011F0881108C090913402992331F081E0A3
:10165000E91204C002C081E001C080E080FD15C035
:101660008091320281110FC08091330281110BC031
:1016700080913402811107C081E09091350291116F
:1016800003C080E001C081E080FD0E94B81A7A8228
:101690009B82FC82ED828E8286E0F801A0E3B2E0BC
:1016A00001900D928A95E1F70E94EA19F82E809137
:1016B0007301F81639F0F09273010E94FA188F2D19
:1016C0000E94D51F80918401843009F055CE83E0BB
:1016D0008093E9008091E80082FF4ECE8091E8007F
:1016E00085FF21C00E944F1281111BC080E2E82EAD
:1016F000F12C480109C08091F100D4018D934D0176
:10170000B1E0EB1AF10869F08091E80085FDF3CFB4
:101710008091E8008B778093E8000E944F12882325
:1017200099F391E001C090E08091E8008B7780937D
:10173000E800992309F420CE2981822F90E0FC0152
:101740003197E331F10508F035C1E557FF4F0C94AF
:1017500098211A828CE09BC08A81823009F450C1A2
:1017600050F4813009F026C10E94FA189B838C83C3
:101770007D836E8321C1833041F0843009F01AC12A
:101780001B821C821D821E8217C16B81DE01149692
:1017900080E090E0262F30E0A901480F591F453026
:1017A000510508F009C1E62FE80FF0E0EC58FE4FB4
:1017B00040814D9301968C31910571F7FDC08A816E
:1017C000823019F0853051F0F5C06B817C818D81BC
:1017D0009E810E949E210E94F719EEC080912802EE
:1017E00080FF03C00E949E1CE7C00E94AD20E4C0A1
:1017F0004C816B818A810E94AE1B9D8308C12D8123
:101800003E813227232732274C816B818A810E94B7
:10181000421BD2C00E94691BCFC08A81813009F06F
:10182000C9C0283099F0293041F18B81813009F00D
:10183000C3C08C81E3E08E9FC00111246FEF70E084
:101840000E944E21862F0E94841CB6C08B8181305D
:1018500029F0823009F0B0C01C82AEC0809128020D
:10186000869586958695FFEF8F9FC001112463E0D2
:1018700070E00E944E216C839FC0809128020E94DC
:101880007E1C9AC05A8298C082E08A8388EE8B833D
:1018900093C0EA80FB80FE24EF24FE248C80912CF0
:1018A0003801C701885E9E4F9301201B310B28151C
:1018B000390508F081C028EEE21622E0F20630F485
:1018C0000E94EC20D30114968C9302C0F301148281
:1018D000FFEFEF1AFF0A2FEF621A720AE2CFEA80D7
:1018E000FB80FE24EF24FE248C80912C3801C7015C
:1018F000885E9E4F9301201B310B2815390508F097
:101900005BC0A8EEEA16A2E0FA0620F4F3016481B7
:101910000E940A21FFEFEF1AFF0A2FEF621A720AE4
:10192000E6CF0E94321B48C084E08A8345C0EA802B
:10193000FB80FE24EF24FE248C80912C3801C7010B
:1019400088969301201B310B28153905A8F5A0EFC7
:10195000EA16F10428F40E94EC20F301848303C00A
:10196000D30114961C92BFEFEB1AFB0AEFEF6E1A2D
:101970007E0AE5CFEA80FB80FE24EF24FE248C80E3
:10198000912C3801C70188969301201B310B281533
:10199000390590F4F0EFEF16F10428F4D301149612
:1019A0006C910E940A21BFEFEB1AFB0AEFEF6E1A4F
:1019B0007E0AE8CF8FEF898340E250E0B80182E0F1
:1019C0000E945B18D9CC80918301882309F4D9CC7B
:1019D000A0E1A9BDB2E1B9BD09B400FEFDCF80917F
:1019E000D8008F7D8093D8008091E0008260809342
:1019F000E0008091E00081FDFCCF0E94921DC1CCEF
:101A000087E290E00E94EC201B821C821D828E8364
:101A1000D3CF2B30310508F076CDAFCD2B3031054B
:101A200008F0C1CDFACD8091860187FF11C0809169
:101A3000E80082FD05C0809184018111F8CF11C0BA
:101A40008091E8008B770BC080918401882349F056
:101A50008091E80080FFF8CF8091E8008E77809336
:101A6000E8000895982F973068F59093E90098174B
:101A700039F07091EC002091ED005091F00003C01E
:101A8000242F762F50E021FD02C09F5FECCF3091D4
:101A9000EB003E7F3093EB003091ED003D7F3093C3
:101AA000ED003091EB0031603093EB007093EC006F
:101AB0002093ED005093F0002091EE0027FDE5CF3C
:101AC00080E008958F708093E90081E0089520916F
:101AD0008C0130918D012617370748F0611571058B
:101AE00039F42091E8002E772093E80001C0B90175
:101AF000FC0120E06115710579F180918401882352
:101B0000F1F18530F1F18091E80083FD3CC08091D6
:101B1000E80082FD2EC08091E80080FFEBCF20918D
:101B2000F3008091F20090E0922B6115710551F065
:101B30008830910538F421912093F10061507109AA
:101B40000196F3CF21E0089709F020E08091E800AA
:101B50008E778093E800CECF2111CFCF0AC080913D
:101B60008401882361F0853061F08091E80083FD75
:101B70000AC08091E80082FFF2CF80E0089582E001
:101B8000089583E0089581E0089543E050E0BC01AA
:101B900084E00E945B18089546E050E0BC0184E0B8
:101BA0000E945B180895AAE2B0E0E9EDFDE00C9414
:101BB000CE21E6E8F1E08EE891E02091F10021935A
:101BC0008E179F07D1F780918701833009F463C096
:101BD00030F4813071F0823009F4A2C0B9C08A308B
:101BE00009F48EC08B3009F46EC0893009F0B0C0A2
:101BF00020C080918601813A09F0AAC08091E80056
:101C0000877F8093E80080918A0190918B01892BD6
:101C100021F468E08AE791E003C060E080E090E0B2
:101C200070E00E94670D8091E8008B778093E80058
:101C30008FC080918601813209F08AC080918A012B
:101C400090918B01009719F0029709F081C0809163
:101C5000E800877F8093E8008091E80082FD05C05E
:101C6000809184018111F8CF73C02091F30080919D
:101C7000F20090E0922B029731F48091F1008130D4
:101C800011F0863021F48091F10080930B01809156
:101C9000E8008B7759C080918601813A09F058C0DD
:101CA00080918A0190918B01892B09F051C080911C
:101CB000E800877F8093E8008091E80080FFFCCFF8
:101CC00080910C013CC080918601813209F040C0B6
:101CD00080918A0190918B01892BD1F58091E80048
:101CE000877F8093E8000E94130D81E09091880126
:101CF000911101C080E080930C010E94921D28C0C8
:101D000080918601813221F58091E800877F809360
:101D1000E8000E94130D8091890180930A0118C088
:101D200080918601813AA1F48091E800877F8093B9
:101D3000E8008091E80080FFFCCF80910A01809349
:101D4000F1008091E8008E778093E8000E94130DE7
:101D50008091E80083FFE7C180918601909187011F
:101D6000492F50E04A30510508F0DDC1FA01E25632
:101D7000FF4F0C949821803821F0823809F0D3C1AC
:101D800008C08091820190918301992389F082603B
:101D90000FC080918A018F70873008F0C4C1809392
:101DA000E9008091EB0085FB882780F91092E9001B
:101DB0009091E800977F9093E8008093F100109253
:101DC000F10071C1282F2D7F09F0ADC1882319F0D2
:101DD000823061F0A8C180918801813009F0A3C1EF
:101DE000933009F080E0809383012EC080918801B8
:101DF00081112AC080918A018F702FEF280F263021
:101E000008F091C18093E9002091EB0020FF1CC0F5
:101E1000933021F48091EB00806214C09091EB002C
:101E200090619093EB0021E030E0A90102C0440FE3
:101E3000551F8A95E2F74093EA001092EA008091DC
:101E4000EB0088608093EB001092E9008091E8003D
:101E5000877F8093E8000E94130D65C1811163C1E3
:101E6000109188011F778091E3008078812B809307
:101E7000E3008091E800877F8093E8000E94130DC3
:101E80008091E80080FFFCCF8091E3008068809320
:101E9000E300111102C082E001C083E0809384015D
:101EA00042C18058823008F03EC1209188013091B3
:101EB00089012C3D53E0350779F583E08A838AE276
:101EC00089834FB7F894DE01139620E03EE051E29B
:101ED000E32FF0E050935700E49120FF03C0E29518
:101EE000EF703F5FEF708E2F90E0EA3010F0C796F2
:101EF00001C0C0968D939D932F5F243149F74FBF4A
:101F00008091E800877F8093E8006AE270E0CE016C
:101F100001960E94670DB5C080918A0190918B0156
:101F2000432F552743305105A9F068F4413051053E
:101F300009F408C14230510509F0F5C08BE590E085
:101F4000ECE1F3E04BC04132510529F14232510539
:101F500089F1E9C0C901992781309105A1F058F0B4
:101F6000029709F0E0C0E9E8F3E0E4918E2F90E0F9
:101F7000E9E8F3E030C0EDEBF3E0E4918E2F90E080
:101F8000EDEBF3E028C0EBE9F3E0E4918E2F90E075
:101F9000EBE9F3E020C08330910508F0C4C0880F5E
:101FA000991FFC01EE5DFE4F0190F081E02D89E06C
:101FB00090E014C08330910508F0B5C0FC01EE0F2D
:101FC000FF1FE45EFE4F0190F081E02DDC01A75E73
:101FD000BE4F8C9190E0009709F4A5C02091E800D5
:101FE000277F2093E80020918C0130918D0182178A
:101FF000930708F49C0140E02115310589F1809197
:102000008401882309F43DC08530D9F18091E8002E
:1020100083FD37C08091E80082FD2FC08091E800E9
:1020200080FFEACF4091F3008091F20090E0942B82
:102030002115310559F08830910540F444914093C1
:10204000F1003196215031090196F2CF41E0089715
:1020500009F040E08091E8008E778093E800CCCFD3
:102060004111CDCF0AC080918401882351F0853081
:1020700041F08091E80083FD04C08091E80082FF78
:10208000F2CF8091E8008B778093E8004CC08038D5
:1020900009F049C08091E800877F8093E800809133
:1020A00085018093F1008091E8008E77D2CE811176
:1020B0003AC08091880190918901992702979CF5F7
:1020C0008091E800877F8093E80010918801109349
:1020D00085010E94130D111106C08091E30087FD58
:1020E00002C081E001C084E08093840142E061ECA1
:1020F00081E00E94320D42E261EC84E00E94320DE8
:1021000042E261EC82E00E94320D42E260EC83E048
:102110000E94320D80918401843011F081E001C071
:1021200082E080930D018091E80083FF10C08091D0
:10213000E800877F8093E8008091EB0080628093C5
:10214000EB0005C082E190E0E7E7F3E047CFAA9615
:10215000E3E00C94EA211F920F920FB60F92112424
:102160002F933F934F935F936F937F938F939F939F
:10217000AF93BF93CF93DF93EF93FF93C091E900A9
:10218000CF708091EC00D82FD17080FDD0E81092F4
:10219000E9008091F000877F8093F00078940E949E
:1021A000D30D1092E9008091F00088608093F000D8
:1021B000CD2BCF70C093E900FF91EF91DF91CF91CC
:1021C000BF91AF919F918F917F916F915F914F914F
:1021D0003F912F910F900FBE0F901F901895E8ED33
:1021E000F0E080818E7F80831092E2001092DA000E
:1021F0001092E100A0EEB0E08C9181608C93808120
:102200008F77808319BCA7EDB0E08C918E7F8C9383
:1022100080818F7E8083109279010895A0E0B0E0E4
:10222000E4E1F1E10C94C921C8EDD0E088818F7E12
:102230008883E7EDF0E080818160808384E082BF65
:1022400081E08093790188818E7F888302EE10E09F
:10225000F80110821092DA0081EEC82ED12CF6011E
:10226000108288818F7788838881806888838881BD
:102270008F7D888319BC1092840110928501109281
:1022800083011092820190EEE92EF12CF7018081FA
:102290008B7F808388818160888342E060E080E07A
:1022A0000E94320DF60180818E7F8083F80180814B
:1022B00081608083808188608083F70180818E7F48
:1022C0008083888180618883CDB7DEB7E8E00C9495
:1022D000E5211F920F920FB60F9211242F933F9377
:1022E0004F935F936F937F938F939F93AF93BF931E
:1022F000EF93FF938091E10082FF09C08091E2009B
:1023000082FF05C08091E1008B7F8093E100809186
:10231000DA0080FF2AC08091D80080FF26C080911B
:10232000DA008E7F8093DA008091D90080FF18C098
:1023300080E189BD82E189BD09B400FEFDCF81E065
:10234000809384018091790181110FC00E94EF1068
:102350000E940E118091E20084608093E20005C02B
:1023600019BC10928401109279018091E10080FFE4
:102370001AC08091E20080FF16C08091E2008E7F3B
:102380008093E2008091E20080618093E20080917E
:10239000D80080628093D80019BC85E080938401C6
:1023A00083E080930D018091E10084FF37C080912C
:1023B000E20084FF33C080E189BD82E189BD09B4B8
:1023C00000FEFDCF8091D8008F7D8093D800809152
:1023D000E1008F7E8093E1008091E2008F7E809308
:1023E000E2008091E20081608093E20080918501AB
:1023F000882311F084E007C08091E30087FD02C0CC
:1024000081E001C083E08093840180918401843065
:1024100011F081E001C082E080930D018091E10024
:1024200083FF2CC08091E20083FF28C08091E100EF
:10243000877F8093E10082E0809384011092850180
:102440008091E1008E7F8093E1008091E2008E7F99
:102450008093E2008091E20080618093E20042E09C
:1024600060E080E00E94320D8091F00088608093EF
:10247000F00081E080930D0180930C01FF91EF91BA
:10248000BF91AF919F918F917F916F915F914F918C
:102490003F912F910F900FBE0F901F901895209194
:1024A000E4003091E50095E64091EC00842F8170C6
:1024B00040FF23C08091E80080FD1DC08091840111
:1024C000882399F0853099F08091EB0085FD11C04B
:1024D0004091E4005091E5002417350729F391500D
:1024E00011F09A01E1CF84E0089582E0089583E03D
:1024F000089581E0089580E008954091E80042FF4A
:10250000DDCF089580E0089590913F0292FF10C0C2
:1025100041E0282F2471243009F040E031E0282FD9
:102520002871283009F030E0431711F02CE08227A1
:1025300093FF10C041E0282F2471243109F040E0BE
:1025400031E0282F2871283109F030E0431711F0CD
:102550002CE082273091400230FF10C051E0282F3C
:102560002171213009F050E041E0282F28712830F6
:1025700009F040E0541711F029E0822731FF10C024
:1025800041E0282F2171213109F040E031E0282F6E
:102590002871283109F030E0431711F029E0822733
:1025A00094FD877E08958238910569F1B0F48133F6
:1025B000910509F475C048F48932910509F467C0A2
:1025C0008A32910509F471C008958533910509F4A3
:1025D00059C089339105B9F00895833E910589F179
:1025E00038F4803E9105D1F0823E910529F108959D
:1025F000863E9105C9F1873E9105D9F1843E91054A
:1026000009F06CC027C020913F0220FD57C021FD7A
:1026100055C02091400223FD5BC0089580913F0288
:1026200080FD48C08091400280FF48C080913F02F9
:1026300084FD46C083EE51C080913F0282FF3CC0C2
:10264000F5CF80913F0282FD37C08091400280FD2E
:1026500035C0ECCF8091400281FF36C080913F02AF
:1026600084FD2EC087EE39C080913F0283FF2AC0CF
:10267000F5CF80913F0283FD25C08091400281FD0E
:1026800023C0ECCF80913F0285FD22C01FC0809106
:102690003F0285FD1BC08091400283FF19C00AC024
:1026A00080913F0286FD16C017C080913F0286FDD3
:1026B00013C010C089E311C082EE0FC080EE0DC0C0
:1026C00080E00BC086EE09C084EE07C085E305C03C
:1026D00089E203C08AE201C081E390E0089590910D
:1026E000FA018091D101892B9091D0019923E1F0D9
:1026F000892B90910C01913041F490913F0297FF0A
:1027000004C09EE12AE032E003C096E022E032E01D
:10271000F90120E0915028F031913323D9F32F5F54
:10272000F9CF21111092D00108952091CE019091FE
:10273000950157E02917A9F030E0529FF001539F0F
:10274000F00D1124EA56FE4F7181761306C0708198
:10275000781303C07581741306C02F5F3F4F277035
:10276000E9CF80E0089581E00895F894E82FE2959C
:10277000EF70F0E031A1282F2F7081E090E001C0D0
:10278000880F2A95EAF7982F9095932391A392A109
:10279000892B82A378940895A5E0B0E0E2EDF3E1FF
:1027A0000C94C621AE014F5F5F4F7A0185E0FA01BC
:1027B00011928A95E9F70EE011E06A01AA24A39428
:1027C000B12CF80180818F3F09F441C0F894E82FC3
:1027D000E295EF70F0E021A18F70A50102C0440FD7
:1027E000551F8A95E2F7CA01922F982B91A392A1C7
:1027F0008095892382A3789400C0E3E1F1E0912CD5
:1028000031E021912F3F89F0A22FA295AF70B0E067
:1028100090968C9190E02F7002C0959587952A959F
:10282000E2F780FD02C0832F01C080E0982A330FB9
:1028300051E0E931F50729F7F80180818F3F11F068
:102840000E94B513F0EAFA95F1F7F60190820F5F56
:102850001F4FFFEFCF1ADF0A41E00331140709F0E1
:10286000B0CF45E050E0B70186E691E00E94F62146
:10287000892B91F085E0F701A6E6B1E001900D9279
:102880008A95E1F781E08093FF010E9406199093F9
:10289000FE018093FD010CC08091FF01882341F06F
:1028A0008091FD019091FE010E94EB18059710F4B4
:1028B00080E018C045E050E066E671E084E791E012
:1028C0000E94F621892B59F085E0E6E6F1E0A4E7C5
:1028D000B1E001900D928A95E1F781E001C080E0BE
:1028E0001092FF012596EBE00C94E221753048F43C
:1028F000663038F4843028F4462F672F0E94AE1BD0
:10290000089580E090E008951F93CF93DF930E9495
:10291000D312EC01C11580E5D807E8F5C11590E4A4
:10292000D90708F0A8C0C03ED10530F5CD3CD1058F
:1029300008F094C0C83AD10578F4C53AD10508F03A
:1029400083C0C130D10509F47CC008F4F2C0C430A2
:10295000D10508F0F1C0EDC0C33CD10508F0E9C0D5
:10296000C85AD0E0CC0FDD1FC55DDE4F0990D8817D
:10297000C02DCE019464E1C0C11580E2D80708F0F3
:10298000CBC0C11591E0D90708F06BC0C83ED10596
:1029900008F4D2C0CEC0C03682E5D80728F5C034CE
:1029A00092E5D90708F079C0C03282E5D80708F06F
:1029B0006CC0C11592E5D90708F481C04C2F46952B
:1029C000469580E2489FA0011124C37021E030E0C9
:1029D000C90102C0880F991FCA95E2F7EA01C82B06
:1029E000D92BCE019D68A9C0C03A82E5D807B8F4BA
:1029F0008C2F8F71C03892E5D90708F07BC086957F
:102A0000869590E2899F90011124C37081E090E047
:102A100002C0880F991FCA95E2F79A6868C0C03C47
:102A200082E5D80708F46DC0C03E92E5D90708F0EA
:102A300080C0CF71DD27DC2FCC27CE01806F906A5C
:102A40007CC081E090E079C0C55AD0E0C85DDE4F1F
:102A50008881C82FD0E0CE0190646FC0CE01906510
:102A60006CC08D2F0E948412182FCE0199270E94CE
:102A7000D3121F715CC0CE0199270E94D312CC27BC
:102A8000DF70D06A8C2B9D2B58C0CF71D0E0DC2F2B
:102A9000CC27CE01816F906A50C08C2F8F718695A4
:102AA000869590E2899F90011124C37081E090E0A7
:102AB00002C0880F991FCA95E2F79C6818C08C2F36
:102AC0008F710E94841295E0D695C7959A95E1F78B
:102AD000CF70D0E0DC2FCC27282F30E084FF05C05A
:102AE00084E0220F331F8A95E1F7D069CE01822B53
:102AF000932B23C090E0D82FCC27CE01846F906A0F
:102B00001CC08C2F8F710E9484128F7190E0D82F7F
:102B1000CC27CE01906211C08D2F8F710E9484123C
:102B2000182FCE0199270E94D3121F719062912B0A
:102B300004C080E090E001C0CE01DF91CF911F91F1
:102B40000895A6E0B0E0E7EAF5E10C94CD210E94FB
:102B500006198C018091FB019091FC01081719075F
:102B600081F019821A820E940619682F49815A81C0
:102B7000792F80E090E00E9407201093FC010093E1
:102B8000FB012696E4E00C94E92180959091FA01EE
:102B900089238093FA01089580910C01813051F5C9
:102BA00080913F0287FF26C00E946F138093090225
:102BB00040E250E062ED71E088E092E00E94F62190
:102BC000892BD9F180E2E8E0F2E0A2EDB1E00190DA
:102BD0000D928A95E1F7E0913B02F0913C0230972B
:102BE00061F186E0809308020480F581E02D88E0A1
:102BF00092E022C00E946F138093000248E050E0F0
:102C000062EF71E080E092E00E94F621892BA9F04A
:102C100088E0E0E0F2E0A2EFB1E001900D928A9549
:102C2000E1F7E0913B02F0913C02309731F00280F5
:102C3000F381E02D80E092E0099508959091CF0115
:102C4000809589238093CF01282F277069F49817E6
:102C500059F09091400292FF07C08695869586951F
:102C60000E94531D1092CF0108959091400292FB53
:102C7000222720F9281779F080FB92F990934002DF
:102C800060913F027091400284E090E00E94282110
:102C900082E00E941E1608958091CE0190919501C8
:102CA000891719F08F5F8770FBCF0895CF93DF935B
:102CB0008091940182958F7009F04EC080919301AC
:102CC000882309F449C08091CE014091950150912B
:102CD0008F0160918E01C0919001D091910177E0B8
:102CE0008417D1F190E0789FF001799FF00D1124C5
:102CF000DF01AA56BE4F14962C911497222349F156
:102D000011962C911197251324C02C91261321C0C4
:102D100015962C91159721111CC012962D913C915E
:102D200013972C1B3D0B283C310598F4809194019E
:102D30008F70806180939401E456FE4F80818F7084
:102D4000806180838EE891E00E9478020E944C1698
:102D500003C001968770C4CFDF91CF910895A4E19D
:102D6000B0E0E5EBF6E10C94C5218C0186E0F801BA
:102D7000DE011F9601900D928A95E1F7F80184819A
:102D8000E5809EE8892E91E0992E90919201911113
:102D900020C0882309F463C1EE2009F442C0C801B1
:102DA0000E946F1DF82E8823E1F187E0F801D4011D
:102DB00001900D928A95E1F780919201813031F472
:102DC00080918E0190918F010E94DA1C0E9456160C
:102DD00048C1F801D080C180A280B380F0909301F7
:102DE0002091900130919101FF2009F4E7C0A501E5
:102DF000421B530B483C510508F09DC0882309F441
:102E000030C180919401282F207F90918F0122233F
:102E100061F09C1509F460C0C8010E946F1D81110A
:102E200063C0C8010E9478021AC19C1113C090911E
:102E30008E019D110FC0E1100DC08F7080618093D5
:102E400094018EE891E00E94780280919401F8014B
:102E5000868303C1E1103AC040E06C2D8D2D0E94A5
:102E6000951340E06C2D8D2D0E949513E82E811155
:102E7000F4C0DF86C88A8F8598890E94DA1C292FC2
:102E800022952F70243020F49F70223028F009C042
:102E90002A50223080F014C0992349F0811107C0D4
:102EA00013C0992321F0F8019681907F69F0805E2C
:102EB000883030F409C0803F38F0815F833020F0E3
:102EC000C8010E947802EF2CFE2CCBC080919401A7
:102ED000816080939401C1C090918E019D119CCF1F
:102EE000E1109ACFF80198C0EE2009F49ACF209112
:102EF0009401822F82958F7090E002978CF08091E0
:102F00008E0190918F0199878887BB86AA868091D0
:102F100092018C871D862E87CE0108960E9478022A
:102F200087E0F801AEE8B1E001900D928A95E1F7F3
:102F30000E94561694C090919401292F207F51F43D
:102F40008EE891E00E94780287E0F40111928A9560
:102F5000E9F783C0882309F484C080918F018C1124
:102F60000CC080918E018D1108C0E11006C0F801DF
:102F70009683C8010E9478026AC0C8010E946F1D32
:102F8000882309F44ECFEE2009F44BCF2091940111
:102F9000822F82958F7090E0029714F280918E01BB
:102FA00090918F019A838983BC82AB828091920138
:102FB0008D831E822F83CE010196B0CFA21AB30A51
:102FC000F8ECAF16B10408F042C0882309F447C0FA
:102FD000FE2CEE2009F425CF80918F018C1129C0A1
:102FE00080918E018D1125C09091940190FD18C0A3
:102FF000892F82958F70282F30E02115310581F0BF
:10300000F80196832F30310541F08F5F982F92950C
:10301000907F86818F70892B8683C8010E947802F9
:1030200087E0F801AEE8B1E001900D928A95E1F7F2
:1030300018C0C8010E946F1D811172CF8091940148
:10304000816080939401C8010E9478020AC087E0E1
:10305000F40111928A95E9F704C0F12C02C0FF2413
:10306000F3948F2D6496ECE00C94E12190916C0127
:1030700021E030E0F90101C0EE0F8A95EAF7D901AD
:1030800002C0AA0FBB1F6A95E2F7BD016E2B01C0FB
:10309000220F4A95EAF7892F8623681303C0892FE8
:1030A000822B03C02095822F89230E94501D0895F2
:1030B00080910B0108950F931F93CF93DF938B01A2
:1030C000EA0190918401943079F58F708093E90042
:1030D0008FEF9091E800815095FD06C095ED9A958F
:1030E000F1F700008111F5CF8091E80085FF1CC049
:1030F0000E944F12882361F08091E8008E778093C0
:10310000E80012C0F80181918F018093F1002197AE
:10311000209791F38091E80085FDF4CF8091E8003D
:103120008E778093E800E4CFDF91CF911F910F91CC
:10313000089540E250E0BC0184E00E945B180895CD
:10314000CF93DF93EC0148E050E0BC0181E00E94A6
:103150005B1888E0FE01AAE7B1E001900D928A9524
:10316000E1F7DF91CF91089587E797E79093010802
:10317000809300089AE088E10FB6F894A8958093B0
:1031800060000FBE90936000FFCF78941F920F9263
:103190000FB60F9211248F939F93AF93BF9380919B
:1031A000420290914302A0914402B09145020196DF
:1031B000A11DB11D8093420290934302A09344024B
:1031C000B0934502BF91AF919F918F910F900FBE29
:1031D0000F901F9018959C014FB7F8948091420270
:1031E00090914302A0914402B09145024FBF821BCF
:1031F000930B08952FB7F8946091420270914302A7
:1032000080914402909145022FBF08952FB7F89402
:103210008091420290914302A0914402B0914502F4
:103220002FBF08951F920F920FB60F9211248F9304
:103230009F93AF93BF9380914102811113C08091FE
:10324000420290914302A0914402B09145024196FE
:10325000A11DB11D8093420290934302A0934402AA
:10326000B0934502BF91AF919F918F910F900FBE88
:103270000F901F90189590910C01913021F490912E
:103280003F0297FD03C0E0E0F2E01DC0E82FE695A5
:10329000E695E695EE31E0F4F0E0E85FFD4F8770EB
:1032A00021E030E0A90102C0440F551F8A95E2F7E2
:1032B000CA0180959281892382830895319652E0D4
:1032C000E630F50729F092818913F8CF1282F6CF04
:1032D000089590910C019130D1F490913F0297FFA5
:1032E00016C0E82FE695E695E695EE3140F5F0E05C
:1032F000E85FFD4F877021E030E0A90102C0440F74
:10330000551F8A95E2F7CA019281892B16C0A2E067
:10331000B2E0EFEF90E02D91821789F0EF3F19F4C2
:10332000211101C0E92F9F5F9630A9F7EF3F39F0D7
:103330000E2E000CFF0BE050FE4F8283089508957F
:10334000A3E0B0E0E6EAF9E10C94CF2120913D0240
:1033500030913E0228173907A1F090933E028093E6
:103360003D02E0913B02F0913C02309751F024E0A5
:1033700029839B838A830084F185E02DCE01019609
:1033800009952396E2E00C94EB21A3E0B0E0EBEC8E
:10339000F9E10C94CF212091390230913A0228179B
:1033A0003907A1F090933A0280933902E0913B02F1
:1033B000F0913C02309751F023E029839B838A836C
:1033C0000084F185E02DCE01019609952396E2E077
:1033D0000C94EB21E0913B02F0913C02309729F0F4
:1033E0000190F081E02D0995089580E0089587E22D
:1033F00090E00E940A210895CF93C82F811102C046
:103400006FEF01C065E284E290E00E940A21C111E1
:1034100002C06FEF01C061E085E290E00E940A21E6
:10342000C11102C06FEF01C064E186E290E00E942A
:103430000A21CF91089584E290E00E94EC20853229
:1034400081F485E290E00E94EC20813051F486E224
:1034500090E00E94EC2091E0843109F090E0892F07
:1034600001C080E0817008950F931F93CF93DF9385
:10347000C42FD22FFC0185818823B1F040933802FC
:103480000E940619909337028093360280E28C0FD7
:10349000883008F068C0C77081E001C0880FCA9505
:1034A000EAF70E94CA1D5FC08091380248133DC0F0
:1034B00080913602909137020E94EB18883C91056A
:1034C000A0F510E21D0FCD17E9F080E28C0F8830D7
:1034D00040F4C77081E001C0880FCA95EAF70E94E6
:1034E000C31D183078F581E09D2F977001C0880FBB
:1034F0009A95EAF70E94CA1D093351F560E570E01C
:1035000089E329C0093319F460E570E002C060E086
:1035100070E0802F0E94BD1F183028F5D77081E021
:1035200001C0880FDA95EAF70AC080E28C0F883074
:10353000D0F4C77081E001C0880FCA95EAF70E94F5
:10354000C31D11C0093351F460E570E089E309C07F
:1035500060E070E0802F0E94BD1FE0CF60E070E06F
:10356000802F0E94BD1FDF91CF911F910F91089571
:103570000E94061920913202211104C020913302C9
:10358000222321F090932F0280932E022091340267
:10359000211104C020913502222321F090932D02A5
:1035A00080932C02E0913B02F0913C02309749F06D
:1035B00082E0809330020680F781E02D80E392E084
:1035C0000995089580912B0280FD16C081FD16C0DB
:1035D00082FD18C080912A02882391F0883290F4ED
:1035E00028E0829FC001112468E270E00E946221FD
:1035F000862F672B29F007C082E0089584E00895A4
:1036000081E0089588E0089580912B0280FD14C028
:1036100081FD14C082FD16C080912902882381F0AB
:103620008E3180F420E5829FC00111246EE170E0AC
:103630000E946221862F089584E1089588E208950A
:1036400088E0089580E50895282F35EB2303C00115
:10365000112497FF03C08058910902C080589F4FE2
:10366000892F0895CF93DF93C8E1D1E060E0CE01C8
:103670000E940A212196C11584E0D807B9F7DF918D
:10368000CF9108951F93CF93DF93962F8430E8F462
:103690006530D8F44630C8F4632F122FC42FD0E021
:1036A000CC0FDD1F2CE0929FC00DD11D11249CE397
:1036B000899FC00DD11D1124CE0188960E940A2138
:1036C000612FCE0189960E940A21DF91CF911F912F
:1036D0000895A0E0B0E0EFE6FBE10C94C721A12C37
:1036E000E12CF12CB12C00E010E0C0E0D0E067014B
:1036F000C00ED11EFE01EE0FFF1FEC0DFD1DEF539E
:10370000FC4F259134914C2F6B2D8A2D0E94421B2A
:103710002196C630D10571F7045F1F4FB39485E041
:10372000B812E3CF8CE3E80EF11CA39484E0A81256
:10373000D9CFCDB7DEB7EAE00C94E32180E00E9458
:10374000FC1960E070E0CB010E94F7190E94691B30
:103750000E94321B81E00E94FC1908950F931F9371
:10376000CF93DF93843008F56530F8F44630E8F401
:10377000C42FD0E0CC0FDD1F2CE0629FC00DD11D07
:1037800011243CE3839FC00DD11D1124CE018896E6
:103790000E94EC2090E0182F0027CE0189960E940D
:1037A000EC209801282BC90102C080E090E0DF9155
:1037B000CF911F910F910895A0E0B0E0E2EEFBE100
:1037C0000C94C521843030F4811105C090918000A3
:1037D0009F7704C083E09091800090689093800070
:1037E000A0918600B0918700282F30E00E94A5218B
:1037F00023E030E040E050E00E9476210027122FC5
:10380000232F342F012F122F232F3327809186004F
:10381000909187006CE070E00E944E216017710764
:1038200030F0C80169E070E00E944E215EC08091D6
:10383000860090918700E0908600F0908700E091EC
:103840008600F0918700C6E0D0E0BE010E944E21C4
:10385000060F171F211D311D4801590185E0880CF5
:10386000991CAA1CBB1C8A95D1F7C701BE010E94F6
:103870004E216F01E12CF12CA7019601260F371F75
:10388000411D511DC501B4010E94762169017A01D3
:10389000E0918600F0918700CA01B9010E943E21A3
:1038A0009B01AC01DF010E94B4219B01AC01C70167
:1038B000B6010E943E21DC01CB012FE0B695A79511
:1038C000979587952A95D1F70091860010918700EA
:1038D00020E030E0081719072A073B0728F4609119
:1038E000860070918700CB01BC01709389006093C2
:1038F0008800CDB7DEB7ECE00C94E121682F86E0BC
:1039000090E00E940A210895843008F083E09091AD
:1039100028029770282F220F220F220F922B9093AC
:103920002802987F21E009F420E09091280220FBF2
:1039300090F9909328020E94DC1B08958091280240
:1039400080FF08C08E7F809328020E947E1C80E04A
:103950000E94DC1B0895CF92DF92FF920F931F937A
:10396000CF93DF936C0100916C0180916B01082B68
:10397000C3E0D0E010E0C8010C2E02C095958795F9
:103980000A94E2F780FD04C02197A8F7F12C09C042
:10399000FC2EB6018C2F0E9476140E94841401978D
:1039A00099F38F2DDF91CF911F910F91FF90DF90B1
:1039B000CF900895CF93DF93EC010E94AB1CBE0122
:1039C0000E9476140E948414DF91CF910895292FCC
:1039D000953078F5863068F590E036E0239F800DCD
:1039E000911D1124682F677023E0969587952A957D
:1039F000E1F7FC01EE0FFF1FE80FF91FEA5BFD4F37
:103A000040E050E080E0219130E0062E02C0369583
:103A100027950A94E2F721703327042E01C0220F64
:103A20000A94EAF7822B4F5F5F4F4330510559F7F5
:103A3000089580E00895292F953088F5863078F52F
:103A400090E036E0239F800D911D1124282F2770D0
:103A500051E001C0550F2A95EAF723E09695879526
:103A60002A95E1F7FC01EE0FFF1FE80FF91FEA5B53
:103A7000FD4F20E030E070E04081CB01022E02C01B
:103A8000969587950A94E2F781708195842785231E
:103A9000842781932F5F3F4F2330310569F70895C5
:103AA00080936C01089521E030E001C0220F8A95D7
:103AB000EAF7209580916C0182230E94501D0895A1
:103AC00021E030E001C0220F8A95EAF780916C0175
:103AD000822B0E94501D089580936B010895FC0174
:103AE00024812223D9F0808191810E94DA1C929551
:103AF0009F70963079F010F4925001C09A50923035
:103B000068F4803F69F018F4883E40F409C0843FAF
:103B100029F406C0883E20F0813F11F080E008952E
:103B200081E008951092FA0180910C01813041F4F6
:103B300080913F0287FF04C08EE1EAE0F2E003C01B
:103B400086E0E2E0F2E0DF011D928A95E9F780E08D
:103B500090E00E94C51980E090E00E94A0191092A8
:103B6000D1010E94CC15E0E3F2E086E0DF011D9276
:103B70008A95E9F71092290210922A0210922B02DC
:103B80000E94B81A0895882321F00E94C5150E944A
:103B9000CC150895882339F09091FA01892B8093F0
:103BA000FA010E94CC150895662309F45CC08D3C8F
:103BB00021F40E94041B819504C08E3C29F40E94CC
:103BC000041B80933302C5C08F3C21F40E94041B68
:103BD000819504C0803D29F40E94041B8093320229
:103BE000B8C0893D19F40E94E21A05C08A3D31F43B
:103BF0000E94E21A819580933402ABC08B3D21F480
:103C00000E94E21A819504C08C3D29F40E94E21AB8
:103C1000809335029EC09FE2980F983078F421E09F
:103C200030E0A90102C0440F551F9A95E2F7CA017E
:103C300090913102892B809331028BC08D3D21F40C
:103C400080912B0281600CC08E3D21F480912B026B
:103C5000826006C08F3D09F07CC080912B02846099
:103C600080932B0276C08D3C39F49091330297FFFC
:103C700035C01092330259C08E3C29F49091330222
:103C80001916BCF32BC0909132028F3C29F497FF98
:103C900025C01092320249C0803D19F41916CCF3A8
:103CA0001DC090913402893D29F41916BCF410927C
:103CB00034023BC08A3D19F497FF10C0F8CF8B3D0A
:103CC00039F49091350297FF09C0109235022DC04A
:103CD0008C3D21F4909135021916BCF39FE2980FA8
:103CE000983080F421E030E0A90102C0440F551F54
:103CF0009A95E2F7CA0180959091310289238093C9
:103D0000310213C08D3D21F480912B028E7F0BC0B8
:103D10008E3D21F480912B028D7F05C08F3D29F4CB
:103D200080912B028B7F80932B0280913202811134
:103D300006C080913302811102C010922902809145
:103D40003402811106C080913502811102C01092A7
:103D50002A020E94B81A0895882309F456C08238AE
:103D600059F40E94EA1981FF50C089E30E94691941
:103D70000E94CC1589E30CC0833879F40E94EA19BB
:103D800080FF43C083E50E9469190E94CC1583E53A
:103D90000E943B190E94CC150895843859F40E9462
:103DA000EA1982FF32C087E40E9469190E94CC158B
:103DB00087E4EECF9CEF980F913A50F390E2980F82
:103DC000983050F4877091E001C0990F8A95EAF716
:103DD000892F0E94C515DECF9BE5980F933028F4FC
:103DE00080E090E00E94C519089598E5980F9B31F6
:103DF00028F480E090E00E94A019089593E3980FC2
:103E0000933118F460E00E94D41D0895CF93882365
:103E100009F4B1C0C82F8238A1F40E94EA1981FDCB
:103E2000AAC089E30E9469190E94CC152FEF87EE82
:103E300093E0215080409040E1F700C0000089E30A
:103E400015C08338C1F40E94EA1980FD94C083E54F
:103E50000E9469190E94CC152FEF81EE94E0215049
:103E600080409040E1F700C0000083E50E943B19CC
:103E70000E94CC1580C08438A1F40E94EA1982FD0A
